:0200000480007A
:10000000171800001308480097180000938888000C
:10001000930100008320080003214800171A000004
:10002000130A4AFE970A0000938A4A0183270A00AE
:1000300023A0FA000F1000003701000023A01800D1
:1000400023A2280023A4380023A6F80017150000D7
:10005000130545FC971500009385C5FC370610F085
:100060001306C6F26306B5028326C5002320D60018
:10007000832685002320D600832645002320D60032
:10008000832605002320D600130505016FF09FFD90
:10009000370510F0130505F22320050000000000CD
:0400A000000000005C
:10100000B3011100300000001200000000000000D9
:10101000FFFFFFFFFFFFFFFFFFFFFFFFFFFFFFFFE0
:040000058000000077
:00000001FF
